:020000040000FA
:060000005FEF0DF012009D
:061000005FEF0DF012008D
:0610080087EF0BF012005F
:061018006BEF0CF012006A
:06102A000200DA1A0000CA
:101030006A0000000A000000D61A000074000000D8
:0410400004000000A8
:0C104400800E6F6EE00E6E14800801E05C
:10105000FBD7706A709E708C040E7010706E718E6B
:10106000719A71987186719471927180729E729C5E
:10107000729472927280776A779E778C608C609A95
:101080000D01FC6BA46A030EA36EA56EFA696F6A6C
:10109000E00E6E1401E0FCD71200A450020B06E132
:1010A000A450020B03E1A450010B47E060AE06D050
:1010B000000E77141009776E41D839D00F0150AF68
:1010C00006D0000E77141109776E38D830D00E0193
:1010D00020AF06D0000E77141209776E2FD827D0D4
:1010E00030AF06D0000E77141309776E27D81FD0C3
:1010F00040AF06D0000E77141409776E1FD817D0B2
:1011000050AF06D0000E77141509776E17D80FD0A0
:1011100060AF06D0000E77141609776E0FD807D08F
:1011200070AF05D0000E77141709776E07D8A4B2F8
:10113000A492A4B2A492A4B0A4901200D9CFE6FFC6
:10114000E1CFD9FF0F0EE1266250080B02E1000E3D
:1011500001D0010EE76E040EE7CFDBFFDE6ADE6A28
:10116000DE6ADD6ADD52DD52DB046FE16150006E44
:10117000016A026A036A150E1F0B07E0D890003659
:10118000013602360336E806F9E1E00E6214046E19
:10119000056A066A076A0D0E1F0B07E0D890043631
:1011A000053606360736E806F9E1045000260550F4
:1011B00001220650022207500322030E6214086E19
:1011C000096A0A6A0B6A100E1F0B07E0D8900836EE
:1011D00009360A360B36E806F9E1085000260950B0
:1011E00001220A5002220B50032263500C6E0D6A3A
:1011F0000E6A0F6A080E1F0B07E0D8900C360D36EA
:101200000E360F36E806F9E10C5000260D5001228B
:101210000E5002220F5003226450106E116A126A9F
:10122000136A10500026115001221250022213504E
:10123000032200C0DFFF010E01C0DBFF020E02C06F
:10124000DBFF030E03C0DBFF2FD06150006E016A8D
:10125000026A036A030E1F0B07E0D89000360136BE
:1012600002360336E806F9E16250046E056A066A42
:10127000076A050ED8900732063205320432E806B6
:10128000F9E10450002605500122065002220750C1
:10129000032200C0DFFF010E01C0DBFF020E02C00F
:1012A000DBFF030E03C0DBFF6550010B026E6550D0
:1012B000020B01E0010EE824016E6550040B01E011
:1012C000010E040DF3CF00F06550080B01E0010E94
:1012D000080DF350002401240224E76E060EE7CF28
:1012E000DBFF6550400B02E1000E01D0010EE76EFE
:1012F000050EE7CFDBFF070E66CFDBFF080E67CFDB
:10130000DBFF090E68CFDBFF0A0E69CFDBFF0B0E98
:101310006ACFDBFF0C0E6BCFDBFF0D0E6CCFDBFF5C
:101320000E0E6DCFDBFF609ED9CFE9FFDACFEAFF6B
:10133000EECFE6FFEECFE6FFEECFE6FFEECFE6FF25
:10134000EECFE6FFEECFE6FFEECFE6FFEECFE6FF15
:10135000EECFE6FFEECFE6FFEECFE6FFEECFE6FF05
:10136000EECFE6FFEECFE6FFEECFE6FF7CEC0CF033
:10137000006E0F0EE15E00500F0EE15C02E2E16ACA
:10138000E552E16EE552E7CFD9FF1200D9CFE6FF73
:10139000E1CFD9FF0F0140B704D0000E7714030945
:1013A000776E0F0130B704D0000E77140409776E02
:1013B0000F0120B705D0000E77140509776E02D013
:1013C000000EE4D0EF0EDBCF00F000340EE2EF0EA3
:1013D000DBCF01F0030EE76E0118E8AE02D0013456
:1013E00003D0E750D880015402E2EF0EDB6AF40E1E
:1013F000DB045FE1F00EDBCF00F0F10EDBCF01F09C
:10140000F20EDBCF02F0F30EDBCF03F0150ED89017
:101410000332023201320032E806F9E10050616E17
:10142000F00EDBCF05F0F10EDBCF06F0F20EDBCFD6
:1014300007F0F30EDBCF08F00D0ED890083207321C
:1014400006320532E806F9E1E00E0514046EF00EEE
:10145000DBCF00F0F10EDBCF01F0F20EDBCF02F0BC
:10146000F30EDBCF03F0100ED890033202320132BC
:101470000032E806F9E1030E00140424626EF00E57
:10148000DBCF00F0F10EDBCF01F0F20EDBCF02F08C
:10149000F30EDBCF03F0080ED89003320232013294
:1014A0000032E806F9E10050636EF00EDB50646E26
:1014B0002FD0F00EDBCF00F0F10EDBCF01F0F20EFB
:1014C000DBCF02F0F30EDBCF03F0030ED890033234
:1014D000023201320032E806F9E10050616EF00E8E
:1014E000DBCF00F0F10EDBCF01F0F20EDBCF02F02C
:1014F000F30EDBCF03F0050E1F0B07E0D89000368C
:10150000013602360336E806F9E1E00E0014626E99
:10151000656AF60EDB50080803E2080E656E03D01C
:10152000F60EDB50656EF50EDB0402E1658C01D032
:10153000659CF70EDB50666EF80EDB50676EF90E99
:10154000DB50686EFA0EDB50696EFB0EDB506A6E84
:10155000FC0EDB506B6EFD0EDB506C6EFE0EDB5036
:101560006D6EF40EDB0402E1010E01D0000EE8B056
:101570006286E8A06296EF0EDBCFE6FFFC0E6014F9
:10158000E552E710606E6086010E00D0E552E7CFAD
:04159000D9FF12006D
:0C159400D9CFE6FFE1CFD9FF0F0EE12612
:1015A000A3D922EC08F03DEC0DF047EC0DF0000162
:1015B0006C51185C006E6D511958016E6E511A58BD
:1015C000026E6F511B58036EF40E005C010E015841
:1015D000000E0258000E035801E28ED047EC0DF0C9
:1015E00018C06CF019C06DF01AC06EF01BC06FF01F
:1015F000660EDE6E060EDE6EDE6ADD6ADD52DD52DE
:10160000040EDB6A050EF36E060EF3CFDBFF480E09
:10161000F36E070EF3CFDBFF00016A51E76E080E91
:10162000E7CFDBFF000E6A15006EFF0E6B15016E33
:10163000D89001320032090E00C0DBFF6AC003F00F
:101640006BC004F0056A036A046A020E1F0B03C034
:1016500000F004C001F005C002F006E0D8900232AC
:1016600001320032E806FAE10A0E00C0DBFF6AC070
:1016700000F06BC001F0026A036A006A016A026A44
:10168000030ED8900332023201320032E806F9E14B
:101690000B0E00C0DBFF00016A2B000E6B23010E56
:1016A000E66ED9CFE9FFDACFEAFFEECFE6FFEECF65
:1016B000E6FFEECFE6FFEECFE6FFEECFE6FFEECFA2
:1016C000E6FFEECFE6FFEECFE6FFEECFE6FFEECF92
:1016D000E6FFEECFE6FFEECFE6FFEECFE6FFEECF82
:1016E000E6FFEECFE6FFC6EC09F0006E100EE15EFD
:1016F0000050000901E1D3D758D70F0EE15C02E298
:10170000E16AE552E16EE552E7CFD9FF1200DACF88
:10171000E4FFE2CFDAFFE9CFE4FFEACFE4FFF6CF60
:10172000E4FFF7CFE4FFF5CFE4FFF3CFE4FFF4CF1E
:10173000E4FFFACFE4FF00EE14F00B0EE80403E33D
:10174000EECFE4FFFBD700EE00F0140EE80403E355
:10175000EECFE4FFFBD7E652D9CFE6FFE1CFD9FFCA
:101760000F0EE1264DEC08F0F250100B01E184D091
:10177000F250020B01E180D047EC0DF000017051F6
:10178000185C1F6E71511958206E72511A58216ED3
:1017900073511B58226ED880320E1F54000E2054F5
:1017A000000E2154000E225466E28272910EDE6E0B
:1017B000DE6ADE6E1F0EDD6EDD52DD52010EF36E4F
:1017C000040EF3CFDBFF010EF36E050EF3CFDBFF4C
:1017D000010EF36E060EF3CFDBFF010EF36E070E64
:1017E000F3CFDBFFF36E080EF3CFDBFF090EF36ED2
:1017F000F3CFDBFF080EF36E0A0EF3CFDBFF030E11
:10180000F36E0B0EF3CFDBFF010EE66ED9CFE9FFCF
:10181000DACFEAFFEECFE6FFEECFE6FFEECFE6FF50
:10182000EECFE6FFEECFE6FFEECFE6FFEECFE6FF30
:10183000EECFE6FFEECFE6FFEECFE6FFEECFE6FF20
:10184000EECFE6FFEECFE6FFEECFE6FFEECFE6FF10
:10185000C6EC09F01F6E100EE15E1F50000901E199
:10186000D3D747EC0DF018C070F019C071F01AC052
:1018700072F01BC073F0F29251EC0DF00F0EE15CB0
:1018800002E2E16AE552E16EE552E7CFD9FFE552A7
:1018900000EE13F0140EE80403E3E5CFEDFFFBD7F1
:1018A00000EE1EF00B0EE80403E3E5CFEDFFFBD7DF
:1018B000E5CFFAFFE5CFF4FFE5CFF3FFE5CFF5FF86
:1018C000E5CFF7FFE5CFF6FFE5CFEAFFE5CFE9FF8C
:1018D000E5CFDAFF1100DACFE4FFE2CFDAFFE6521C
:1018E000E552E5CFDAFF11009492F19EF28EF28C70
:1018F000F18CF288D08E1200D9CFE6FFE1CFD9FF6C
:10190000D950F00FE96EFF0EDA20EA6E040EEE18E1
:1019100006E1030EEE1803E1EE5001E1EE505AE14C
:10192000F70EDB50200801E18282F70EDB50400801
:1019300001E18292F70EDB5080084CE1030EF36E5A
:10194000F00EF3CFDBFF030EF36EF10EF3CFDBFFF0
:10195000F20EDB6AF30EDB6AF40EDB6A010EF36E45
:10196000F60EF3CFDBFF8250020B01E0010EE76EB3
:10197000F70EE7CFDBFF010EE66ED950F00FE96EF0
:10198000FF0EDA20EA6EEECFE6FFEECFE6FFEECFF7
:10199000E6FFEECFE6FFEECFE6FFEECFE6FFEECFBF
:1019A000E6FFEECFE6FFEECFE6FFEECFE6FFEECFAF
:1019B000E6FFEECFE6FFEECFE6FFEECFE6FFEECF9F
:1019C000E6FFC6EC09F0006E100EE15E0050000963
:0C19D00001E1D1D7E552E7CFD9FF1200AA
:0419DC002A0EF66E6B
:1019E000100EF76E000EF86E00010900F550656FDD
:1019F0000900F550666F03E1656701D03DD009002D
:101A0000F550606F0900F550616F0900F550626F85
:101A100009000900F550E96E0900F550EA6E090069
:101A200009000900F550636F0900F550646F090063
:101A30000900F6CF67F0F7CF68F0F8CF69F060C023
:101A4000F6FF61C0F7FF62C0F8FF0001635302E1D7
:101A5000645307E00900F550EE6E6307F8E264078F
:101A6000F9D767C0F6FF68C0F7FF69C0F8FF00014B
:0A1A70006507000E665BBFD7120089
:061A7A00790ED66EFE0E8F
:101A8000D76E070ED56ED58EF284F28A120074C01E
:101A900018F075C019F076C01AF077C01BF000D0AE
:101AA0001200F2A40BD0FE0ED76E790ED66E000196
:0E1AB000742B000E752376237723F294120018
:021ABE001CEE1C
:101AC00000F02CEE00F0F86A1E9CEEEC0CF0CAEC74
:061AD0000AF0FDD7120030
:041AD600000000000C
:061ADA0000000000000006
:041AE0000000000002
:00000001FF
